:1000000010C04AC4CAC428C027C026C025C024C006
:1000100023C022C021C0CEC1A7C51EC01DC01CC0A8
:100020001BC011241FBECFE5D1E0DEBFCDBF10E065
:10003000A0E6B0E0E6E6FEE002C005900D92A03733
:10004000B107D9F721E0A0E7B0E001C01D92A831C7
:10005000B207E1F708D605C7D3CF7F937091C000F0
:10006000072F0170201749F42091C100269577953C
:1000700001E0702700EA202704C02091C1002695E6
:1000800077957093C0002093C1007F9108952FEF62
:10009000F0E02750FFBB60E0E8E6F0E007C02FEF9C
:1000A000F0E02F50FFBB60E0E0E6F0E0E199FECF2A
:1000B0002EBBE09A1DB31F3F29F011936395239542
:1000C0006830A1F7089560C41DC049C079C0B6C0AA
:1000D000ABC1C6C259C4B6C0B5C0B5C0C0C0CCC0A3
:1000E000C8C1EDC1F6C107C21EC228C23FC24AC282
:1000F00089C2DBC200C309C31AC331C33BC352C3A5
:100100005DC39CC36627153529F0103F41F01C3EA6
:10011000F9F034C403E00093710042E034C403E01A
:1001200000937100E0E8F0E0E60F0027F01F37C011
:1001300000E00093C0000093C10000917100013005
:1001400019F0023019F01AC445E01DC446E01BC482
:100150000091C700002319F711C410C40FC43091D7
:10016000710030FF0AC0E8E6F0E0E60F0027F01F5C
:100170002081211711F03E7F79F0E0E6F0E0E60FF4
:100180000027F01F2081211711F03D7F29F03093C7
:100190007100673069F2F6C330937100EFC32081BC
:1001A00000917100033021F0269526950395FACF32
:1001B0002695111F2695111F51E030E444E0E4C359
:1001C000E0E8F0E0E60F0027F01F219100917100B8
:1001D000033029F00130B9F00230E9F0CFC31078D4
:1001E00049F020FDCBC324FD0E7F22FD0D7F00933F
:1001F000710019C021FDC2C324FF0E7F22FF0D7FB5
:100200000093710010C0107819F025FFB7C30BC020
:1002100024FFB4C308C0107819F023FFAFC303C094
:1002200022FFACC300C000917100002309F4A6C3F3
:100230006395603409F0B3CF55277ACF552743E053
:1002400030E0A2C39BC3E8E7F0E0E60F0027F01F11
:100250001083673009F096C391C34BE051E06830DA
:1002600039F0E8E7F0E0E60F0027F01F10818AC3BD
:10027000552784C34CE086C330917100323031F091
:10028000E8E6F0E0E60F0027F01F05C0E0E6F0E04A
:10029000E60F0027F01F0081101759F5613029F093
:1002A000653029F0663029F024C003E0600F6395C3
:1002B0006AC32FEFF0E007E031FD0FE0201BFFBB2A
:1002C000E8E7F0E060E0E199FECF00E00CBB2EBB78
:1002D00011911DBBE29AE19A63952395683099F7D5
:1002E0009F938F93AF93BF931AD0BF91AF918F918C
:1002F0009F9144C3000000000000000008950F9388
:1003000000E806BD00E006BD00E009BF00E40BBF49
:1003100002E003BFBA98C29802E005BF0F91CF93E5
:10032000DF930F931F93FF92EF92B1DEB8DE68E088
:1003300000E0E0E8F0E0A8E6B0E0C0E6D0E09D91A3
:100340008991F92EF094E82EE09438E0092F0823E3
:100350002F2D2E2140E09695441FF694441F86953C
:10036000441FE694441F0695441F2695441F41935D
:100370003A9581F76A9519F700E00093C40000935D
:10038000C3000093C700BB98EF90FF901F910F919F
:10039000DF91CF910895F8940F9300E00093C4008B
:1003A0000093C600009372000093C300BB980F91A6
:1003B000789408950F930FB70F932F93B29927C096
:1003C00000E002BF01E008BF23E008B700FD27C03E
:1003D000B29BFBCF233019F402B70035C0F000E028
:1003E00002BF02B70E31E8F3BA9A02B70238E8F357
:1003F000BA9801E00093C40001E00093C2000093AA
:10040000C300002700937200BB9800E40ABF09B73D
:100410000E7F09BF2F910F910FBF0F9118952A954D
:10042000B1F301E008BFD1CF66271F3011F44DE0D2
:10043000AAC21A3AD9F01A3511F440E1A4C2103F09
:1004400011F441E1A0C2153A11F443E19CC2153800
:1004500009F483CE153711F44AE095C2173A09F42E
:10046000FCCE193709F406CF40E08DC24FE051E0D1
:1004700030C0EBEEF0E0E60F0027F01F639510832D
:10048000623049F008F47FC2633261F0062F0450F5
:100490000093ED0078C20091EB000F71600F0093A4
:1004A000ED0070C20091C00000950093160100910C
:1004B000C1000095009317014EE051E06BE26D32F0
:1004C00039F0EBEEF0E0E60F0027F01F10815AC282
:1004D00055C2633279F0633031F40091EB000F7153
:1004E00023E0020F602FEBEEF0E0E60F0027F01F95
:1004F000108148C243C2633068F4EBEEF0E0E60FCF
:100500000027F01F63950081011739F4633011F063
:1005100031E039C21AEA51E036C20091EE000F779D
:100520000093EE002BC2603019F41093EB002AC246
:100530001093EC0042E151E066270DC06091EB00A2
:100540002091EC0063950027201F21FD0EC0009331
:10055000EC006093EB006091EB006F71EEEEF0E069
:10056000E60F0027F01F10810EC208C2603021F490
:100570001093EB00639507C21093EC0044E151E047
:1005800066270FC06091EB002091EC0001E0600F46
:100590000027201F062F0F7171F02093EC0060934D
:1005A000EB006091EB006F71EEEEF0E0E60F0027DC
:1005B000F01F1081E8C145E162E22091EB0000915B
:1005C000EC00220F001F0330A1F4207C2295E8EC00
:1005D000F0E0E20F0027F01F019100930E0101915E
:1005E00000930F01019100931001019100931101FB
:1005F00009C00FEF00930E0100930F01009310014B
:100600000093110163956D3299F06B3251F40091B2
:10061000C0000095009316010091C1000095009361
:100620001701EBEEF0E0E60F0027F01F1081ABC1E1
:100630006091EB002091EC0001E0600F0027201F8B
:1006400021FD0BC000E00093C0000093C10044E115
:100650002093EC006093EB00A4CF40E0552793C1BA
:1006600066271F3011F446E18EC11A3AD9F01A35C7
:1006700011F449E188C1103F11F44AE184C1153AEF
:1006800011F44CE180C1153809F468CD153711F427
:100690004AE079C1173A09F4E0CD193709F4EACDF7
:1006A00040E071C148E151E030C0EBEEF0E0E60F10
:1006B0000027F01F63951083623049F008F463C18E
:1006C000633261F0062F04500093ED005CC100918D
:1006D000EB000F71600F0093ED0054C10091C0005A
:1006E0000095009316010091C10000950093170139
:1006F00047E151E06BE26D3239F0EBEEF0E0E60FEE
:100700000027F01F10813EC139C1633279F0633098
:1007100031F40091EB000F7123E0020F602FEBEE3C
:10072000F0E0E60F0027F01F10812CC127C16330D5
:1007300068F4EBEEF0E0E60F0027F01F6395008110
:10074000011739F4633011F031E01DC11AEA51E0AC
:100750001AC10091EE000F770093EE000FC16030D8
:1007600019F41093EB000EC11093EC004BE151E033
:1007700066270DC06091EB002091EC006395002787
:10078000201F21FD0EC00093EC006093EB006091F0
:10079000EB006F71EEEEF0E0E60F0027F01F108126
:1007A000F2C0ECC0603021F41093EB006395EBC015
:1007B0001093EC004DE151E066270FC06091EB0013
:1007C0002091EC0001E0600F0027201F062F0F7121
:1007D00071F02093EC006093EB006091EB006F717F
:1007E000EEEEF0E0E60F0027F01F1081CCC04EE1E6
:1007F00062E22091EB000091EC00220F001F033019
:10080000A1F4207C2295EAEDF0E0E20F0027F01F32
:10081000019100930E01019100930F01019100934A
:10082000100101910093110109C00FEF00930E0117
:1008300000930F01009310010093110163956D3235
:1008400099F06B3251F40091C000009500931601AD
:100850000091C100009500931701EBEEF0E0E60F68
:100860000027F01F10818FC06091EB002091EC00F9
:1008700001E0600F0027201F21FD0BC000E0009366
:10088000C0000093C1004DE12093EC006093EB00A9
:10089000A4CF40E0552777C0BB99BA9A2F932FB7C2
:1008A000BB982F930F9305B702600F7E05BF3F9350
:1008B0001F935F933091C3001091700050917200AC
:1008C0000BE402BF09B7016009BF01E008BF55236F
:1008D00099F0332319F446D0552349F020E01795B9
:1008E00010F0BB9A21E0B9DB330FBA9B14C002B7FA
:1008F0000E36E8F3BA980FC002B70735E8F316953D
:1009000021E0B29B02C0106820E0A7DB330F19F48E
:1009100029D05523F1F6BB9901C013C051FD11C078
:10092000B29904C002B7073860F4FACFB29B06C090
:1009300002B7053AB29B02C0C8F303C0BA9ABB988B
:10094000BFCF00E40ABF509372003093C3001093EE
:1009500070005F911F913F910F91BA982F912FBF17
:100960002F911895EF93FF934F936F934091C4008D
:100970006091C500E3E6F0E0E40F0994332740E01E
:10098000552702C0639531E04093C4006093C500D1
:100990006F914F91FF91EF9108951F920F920FB6B3
:1009A0000F9211242F938F939F93AF93BF93C99965
:1009B00018C08091D80081FF14C08091D000909120
:1009C000D100A091D200B091D3000196A11DB11D1C
:1009D0008093D0009093D100A093D200B093D30025
:1009E000C09ACA9918C08091D80082FF14C0809123
:1009F000D4009091D500A091D600B091D700019677
:100A0000A11DB11D8093D4009093D500A093D60072
:100A1000B093D700C09ACB9918C08091D80083FFBB
:100A200014C08091E2009091E300A091E400B091A5
:100A3000E5000196A11DB11D8093E2009093E300B3
:100A4000A093E400B093E500C09ACC9918C08091BF
:100A5000D80084FF14C08091E6009091E700A09137
:100A6000E800B091E9000196A11DB11D8093E60058
:100A70009093E700A093E800B093E900C09ACE9964
:100A800063C08091D80086FF5FC02FEF80E792E0BF
:100A9000215080409040E1F700C00000CE9951C045
:100AA000DD9A2FEF80E792E0215080409040E1F7FF
:100AB00000C000001092D0001092D1001092D2001D
:100AC0001092D3001092D4001092D5001092D6004C
:100AD0001092D7001092E2001092E3001092E4000E
:100AE0001092E5001092E6001092E7001092E800E4
:100AF0001092E9008091C8009091C900A091CA00AD
:100B0000B091CB000196A11DB11D8093C8009093B8
:100B1000C900A093CA00B093CB008091DA009091F5
:100B2000DB00A091DC00B091DD000196A11DB11D9C
:100B30008093DA009093DB00A093DC00B093DD009B
:100B4000DD988AB780618ABF89B38093D80081E03D
:100B50008093EA00BF91AF919F918F912F910F9059
:100B60000FBE0F901F9018951F920F920FB60F9205
:100B700011242F938F939F93AF93BF93EF93FF9382
:100B80008091EA00882309F462C0459B60C08FE031
:100B900097E20197F1F700C00000459B58C0809193
:100BA000CC009091CD00A091CE00B091CF000196E5
:100BB000A11DB11D8093CC009093CD00A093CE00D9
:100BC000B093CF008091CC009091CD00A091CE0049
:100BD000B091CF008093DE009093DF00A093E000FF
:100BE000B093E10080E886BD81E086BDC19A1FBA5E
:100BF00080E090E0282FE199FECF1CBA2EBBFC01CB
:100C0000E853FF4F20812DBBE29AE19A0196803193
:100C1000910581F780E090E020E1280FE199FECF77
:100C20001CBA2EBBFC01E652FF4F20812DBBE29A7D
:100C3000E19A01968031910579F71092EA00C19806
:100C400080E886BD16BCC19A8AB780648ABFFF91CE
:100C5000EF91BF91AF919F918F912F910F900FBE08
:100C60000F901F901895019A4ADB10921201109272
:100C7000130110921401109215011092C8001092E5
:100C8000C9001092CA001092CB001092D0001092AE
:100C9000D1001092D2001092D3001092CC0010928A
:100CA000CD001092CE001092CF001092D40010927E
:100CB000D5001092D6001092D7001092DA00109250
:100CC000DB001092DC001092DD001092E200109226
:100CD000E3001092E4001092E5001092DE00109202
:100CE000DF001092E0001092E1001092E6001092F6
:100CF000E7001092E8001092E90081E08093EA009A
:100D000088B38B6F88BB8BB38FEF8BBBD79ADF9881
:100D1000B99AC198B89AC098D59ADD988BB7806176
:100D20008BBF8EE182BB89B38093D8001FBA80E06D
:100D300090E0282FE199FECF2EBBE09A2DB3FC0165
:100D4000E853FF4F208301968031910591F780E0B1
:100D500090E020E1280FE199FECF2EBBE09A2DB361
:100D6000FC01E652FF4F208301968031910589F7FF
:100D70001092EA0080E090E021E0FC01EE0FFF1FFE
:100D8000EE0FFF1FE853FF4F408151816281738155
:100D90004F3F5F4F6F4F7F4F31F4108211821282AD
:100DA00013822093EA0001968430910531F780E0A8
:100DB00090E021E0FC01EE0FFF1FEE0FFF1FE65257
:100DC000FF4F40815181628173814F3F5F4F6F4F71
:100DD0007F4F31F410821182128213822093EA0035
:100DE00001968430910531F71E9A85B78F7B85BFB8
:100DF000089AD898479888B18B6488B9379880E466
:100E000083B917B8D698969ADE9ADF9A8FEF94E353
:100E10002CE0815090402040E1F700C00000DF98B6
:100E20007894C09B0AC03FE788E391E0315080404E
:100E30009040E1F700C00000C098C19B0AC02FE7B6
:100E400038E381E0215030408040E1F700C00000ED
:100E5000C19885B7806285BF85B78F7E85BF88952D
:060E6000E0CFF894FFCF83
:100E66001D41DA840000058A1D40DA84000005BDB4
:00000001FF
